:020000040000FA
:10000000132800000000090083169B001C141A0826
:1000100083120800C030A0001030A100A10B0E28F0
:10002000A00B0C28080083160313FF239000640024
:1000300081010F30810064000C308500950083122F
:1000400007309900850120300420A80021300420C9
:10005000A90022300420A70030300420B000313045
:100060000420B10032300420AF00A401AC01A20191
:1000700064000A203C203828A30146206620702016
:1000800076209620A0202308850008002408A500DB
:1000900004300505A400250603195128241D542801
:1000A000A6012419A60A080027082602031C6528B1
:1000B000A2186128A21422142808AA002908AB005B
:1000C0000800221CA210221008000800A218221CFE
:1000D0000800AA0B08002B080319A210AB030800A4
:1000E000A21C080023162218231408002C08AD00B7
:1000F00008300505AC002D0603198128AC1D8428A5
:10010000AE01AC19AE0A08002F082E02031C952878
:10011000A2199128A21522153008B2003108B300A7
:100120000800221DA211221108000800A219221D98
:100130000800B20B080033080319A211B30308002A
:0C014000A21D0800A3162219A314080039
:02400E00DC3F95
:06424000500046000300DF
:064260006000EA0003000B
:00000001FF
